:10000000FF2383169000B8280528A000030EA10046
:100010008B12053081000B116400AB0B13281920E3
:1000200055200730AB00210E8300A00E200E8B164A
:100030000900291C3D286400AE0A0319202829283C
:10004000851E26288512FB30AE0029288516FB3038
:10005000AE006400051C2F28051D36285428AA036D
:100060002A08AF0060202F08AA005428AA0A2A08EC
:10007000AF0060202F08AA00542864008516051CD4
:100080004628051D4C28851C52285428AA032608FA
:100090002A02031CAA0A5428AA0A2A082802031CB6
:1000A000AA0354282708AA00003464002A08AC00D8
:1000B0000516B22000000000AC0B5A2805120034CF
:1000C00064302F02031C692864302F0703186C2842
:1000D0006F286430AF006F289B30AF006F2800346A
:1000E000640000307B20A60001307B20A700023096
:1000F0007B20A8000800640083169B001C141A08CB
:100100008312080064008B132F08A70064302F02AD
:10011000A60064302F07A80064002608AD00003058
:100120009A202708AD0001309A202808AD0002303F
:100130009A200800640083169B002D089A001C1565
:100140008B1355309D00AA309D009C141C119C18E7
:10015000A72883120800E830A3006400B220A30B94
:10016000AD280034D630A4000000A40BB42800341D
:10017000831652308100073095000F3085003030F3
:100180009F008312073099008101A201A301A401FD
:10019000A501A601A701A801A901AA01AC01AD0111
:1001A0000730AB00F830AE00AF01850164000530C8
:1001B00081000B118B168B13AB2005182129051913
:1001C00021298518FE28E42864001C30AD00003089
:1001D0009A208030AD0001309A20E430AD0002302A
:1001E0009A2064008516AB208512AB206400051CA4
:1001F000F128051DF128851CF12821296400051C22
:10020000FE28051DFE28702064002708AA008B1711
:10021000AB2064000130A900851809290630A5002B
:100220006400851C0929AB20A50B102964002A084D
:10023000AF0060202F08AA002A08AF008B1382208D
:100240008B1764000230A90070202708AA008B17C2
:0802500064000230A900282916
:084000000000020000000000B6
:02400E00CC3FA5
:064200001C008000E40038
:00000001FF
